:1021FD002020202020200D0A002A4D3A2053656C06
:10220D006674657374206F6B0D0A002A573A20535C
:10221D00656C6674657374206661696C65640D0A1E
:10222D00002A52454144590D0A00000000002A01C0
:10223D00005202007903009E0400C20500E506016C
:10224D00060701270801460901640A01E90F025832
:10225D001403001E03742803C33203F93C04023E29
:100C8D00906EE5EEF0A3EFF0A37401F0906EE7E047
:100C9D00FF6412602AEF75F003A42437F582E43463
:100CAD0022F583E493FC740193FDC3906EE6E09D01
:100CBD00906EE5E09C4008906EE7E004F080CDEF8B
:100CCD0075F003A42437F582E43422F583E493FE12
:100CDD00740193FF906EE5E0FCA3E0FDC3EF9DFF73
:100CED00EE9CFEE4FCFDC8ECC8C9EDC9CAEECACB4A
:100CFD00EFCBA3E075F003A42436F582E43422F59E
:100D0D0083E493FFE4FE1204EDECC0E0EDC0E0EEF1
:100D1D00C0E0EFC0E0906EE7E075F003A42434F579
:100D2D0082E43422F583E493FE740193FFC3906E45
:100D3D00E6E09FFF906EE5E09EFEE4FCFDC8ECC88A
:100D4D00C9EDC9CAEECACBEFCB906EE7E075F003E3
:100D5D00A42439F582E43422F583E493FFE4FE12F2
:100D6D0004EDD0E0FBD0E0FAD0E0F9D0E0F8EF2BC5
:100D7D00FFEE3AFEED39FDEC38FC906EE8120644BC
:100D8D007FE87E037D007C00906EE8E0F8A3E0F93B
:100D9D00A3E0FAA3E0FB1204EDC8ECC8C9EDC9CA83
:100DAD00EECACBEFCB906EE7E0FF75F003A42434D1
:100DBD00F582E43422F583E493FC740193FDEF7521
:100DCD00F003A42437F582E43422F583C374019330
:100DDD009DFFE4939CC313FEEF13FFE4FCFDEB2F8B
:100DED00FFEA3EFEED39FDEC38FCECC0E0EDC0E075
:100DFD00EEC0E0EFC0E0906EE7E0FF75F003A424D5
:100E0D0034F582E43422F583E493FC740193FDEF11
:100E1D0075F003A42437F582E43422F583C37401FD
:100E2D00939DFFE4939CFEE4FCFDF8F9CAEECACB5A
:100E3D00EFCBD0E0FFD0E0FED0E0FDD0E0FC12051E
:020E4D00782209
:10202900201175906F70E05407906EDEF0C3940331
:102039004066E064076061D2117F01122E75E49059
:102049006EDEF07F017D127B03122F3F301706E50C
:102059006860F980397F017D0E7B03122F3F3017AD
:1020690006E56860F980277F017D0A7B02122F3F10
:10207900301706E56860F98015906EDEE004F0E03F
:10208900B403C07F01122F147F0A122E75227F021A
:09209900122F147F0A122E752289
:10153B003012030215D8E56864036009E568640B93
:10154B00600302163DC3E54F78D496FFE54E18961F
:10155B00FE120C8DCBEFCBCAEECAEB4A7003FA7BB3
:10156B0001D201E4906EDEF0CEEACECFEBCF7C0061
:10157B007D0A120436906EDEE024DFF582E4346ED1
:10158B00F583EDF0CEEACECFEBCF7C007D0A1204D3
:10159B0036CAEECACBEFCB906EDEE004F0E0B405BA
:1015AB00C7906EDE7404F0906EDEE0FFF46015748D
:1015BB00DF2FF582E4346EF583E07008906EDEE089
:1015CB0014F080E3EF04906EE4F0D212227F1E122F
:1015DB002E757F017D327B04122F3F30170430169E
:1015EB00FA227F0A122E75906EE4E014906EDEF0F4
:1015FB00906EDEE024DFF582E4346EF583E0700B51
:10160B007F017D0B7B04122F3F8016906EDEE02452
:10161B00DFF582E4346EF583E0FF7D0B7B01122F47
:10162B003F3017043016FA22906EDEE0FF14F0EF15
:03163B0070BE225C
:101F2600D2AF122D3D122E9812000E122D70122FC6
:101F360079122EEE1200031220A2122DFC7BFF7ADC
:101F46002179FD1200C9122EE412299050107BFF50
:101F56007A2279061200C97F01122F14800B7BFFAB
:101F66007A2279181200C9D211121E92906F12E0CD
:101F7600FF12291E122BA212266A906F13E0FEA3EF
:101F8600E0FF1228217BFF7A22792E1200C9C212A5
:101F9600C211301603122CB212153B906F0AE06084
:071FA600F112202980EC225A
:03000B0002218B44
:10218B00C0E0C0F0C083C082C0D075D008C28CAF95
:10219B008CEFFEAD8AED255F78D6F6E55E3E18F640
:1021AB00F58C08E6F58AD28CD56309906F09E0F5BA
:1021BB0063122546D5621B906F09E0F5620561E558
:1021CB006170020560E56145607007E56860037545
:1021DB006805E5686404600F121740122481121C15
:1021EB009B122A9E121DF5D0D0D082D083D0F0D076
:0221FB00E032D0
:10282100E4FCFDFB7AC079A8F81204ED7BE07A2E76
:10283100790078001227DDC374129FF55FE49EF5DD
:102841005E906F09E0F563F562E4F560F561E58995
:1028510054F04401F589758CFF758AFFC2B9D2A97C
:03286100D28C22F4
:0C2EB400906F09E0F562E4F560F5612222
:10266A00E5C520E3FB75C50775C50FE5C530E4FB75
:10267A00AFC6EF75F004A4FFAEF0E5C5C41313545A
:10268A00037C002FF53CEC3EF53BE4F53AE53A25B0
:10269A00E024BFF8A63B08A63CE53C2527F527E53C
:1026AA003B3526F526053AE53AB40AE1E4F539223E
:10174000C0D075D008E5C520E3FBE4F5C575C50834
:10175000F543754401E54364087003021815E5C5B7
:1017600030E4FB85C62885C53DE5436407600EE58A
:10177000C520E3FBE54304F5C54408F5C5E5287538
:10178000F004A4FFAEF0E53DC4131354037C002F16
:10179000F546EC3EF545E54325E02429F8A6450845
:1017A000A646906F08E055446060AF281229C9AF83
:1017B0003D1229C9E543B406088545418546428066
:1017C00049E54364077043E53925E024C0F8C3E5E3
:1017D0002796F527E5261896F526E53925E024BF56
:1017E000F8A64508A646E5462527F527E54535260A
:1017F000F526FEAF277C007D0A1204368E248F2545
:101800000539E539B40A03E4F5390543E54425E033
:10181000F544021755300F1EE4A2C492E4A2C5920B
:10182000E5A29692E6A29792E72568C4F53EAF3E00
:0D1830001229C9853E40C294D294D0D02226
:10226D00C0D075D008300F65906F12E0FD7C0090E6
:10227D006F1AE0FB24FFFFE434FFFE120422EF246B
:10228D0001FFE43EFEC3E51F9FF51FE51E9EF51EF3
:10229D008B3FE53F6021E51EF583E51FF582E0C428
:1022AD0054F02568C4F0906F12E0251FF51FE4353A
:1022BD001EF51E153F80DB906F12E024FFFFE43406
:1022CD00FFFEC3E51F9FF51FE51E9EF51ED0D02214
:0D2EA700E4F576F577F578C2191229572267
:10248100C0D075D008E5686057201954122E6240FB
:102491004F906F12E02404906ED8F0906ED8E060F7
:1024A1003F20133C122A6A8F7512002E0577E577BB
:1024B100700205767004E5766480701CF576F57718
:1024C1000578E578B40C04D2198015122E4FE57801
:1024D10020E0051229578008906ED8E014F080BBE7
:0324E100D0D02236
:102BA200E4906FAEF0A3F0906FAA120650000000FE
:102BB2000074FF78D3F608F6E4906FB0F0F569F58B
:082BC20068906FA974FFF02276
:102D2300C0D075D008756801AF68122DA0C290128B
:0A2D33002EA77F02122F14D0D02229
:102DD000C0D0C291E5612401906FA8F0E435609005
:062DE0006FA7F0D0D02225
:102DE600C0D0C292E5612401906FA8F0E4356090EE
:062DF6006FA7F0D0D0220F
:1012E900C0D075D008E4906ED8F020C604E044015F
:1012F900F020C707906ED8E04402F0906FA9E0FF94
:10130900906ED8E0FE6F603BEE7025906FB6E0FFFF
:101319006005122F1C802C906FB5E0FF64036004F8
:10132900EFB40405122F1C801A7F01122F148013A9
:10133900906ED8E030E0077F01122F1C80057F02F4
:10134900122F1C906ED8E0906FA9F0300B1EA2945A
:10135900300C01B34016C21A122EB4906F06E0FE8B
:10136900A3E0FF122ACE122D2302142A2010030211
:10137900142A906F05E0C4F8540FC868FF906F04F1
:10138900E0C454F048FEC3E54D9FFDE54C9EFCE5E5
:1013990042C4F8540FC868FFE541C454F048FED36D
:1013A900EF9DEE9C4016D21A906FAA1206500000CB
:1013B9000000E4906FAEF0122EB48065C21A906FEF
:1013C900AAE0F8A3E0F9A3E0FAA3E0FBE8C0E0E5AE
:1013D90042C4F8540FC868FFE541C454F048FEC33D
:1013E900EF954DFFEE954CFE3395E0FDFCD0E0F80E
:1013F900EB2FFFEA3EFEE93DFDE83CFC906FAA12A7
:101409000644906F1AE0FF906FAEE004F06F701120
:10141900906F0DE0FEA3E0FF122ACE122D231222B7
:041429006DD0D02290
:101D5400C0D075D008906FAAE0F8A3E0F9A3E0FA28
:101D6400A3E0FBE8C0E0E542C4F8540FC868FFE50F
:101D740041C454F048FEC3EF954DFFEE954CFE333D
:101D840095E0FDFCD0E0F8EB2FFFEA3EFEE93DFDD7
:101D9400E83CFC906FAA120644300E387F007E00A7
:101DA4007D007C00906FAAE0F8A3E0F9A3E0FAA319
:101DB400E0FBD312060A401C906F03E0FFD3E561F9
:101DC4009FE5609400400D122DD0756802AF681233
:101DD4002DA0801A300D17906F18E065617002E530
:101DE40060700B122DD075680AAF68122DA0D0D088
:011DF40022CC
:10211800C0D075D008906FA7E0FEA3E0656170039A
:10212800E5606E7002D291300E3C906F10E0FEA315
:10213800E0FFC3E54F9FFFE54E9EFEC3E5259FE503
:10214800249E5007E4906FAFF0801B906F2BE0FF48
:10215800906FAFE004F06F700D122DE6756803AF55
:1021680068122DA0801A300D17906F19E065617004
:1021780002E560700B122DE675680BAF68122DA092
:03218800D0D02292
:102CD000C0D075D008906FA7E0FEA3E065617003D7
:0C2CE000E5606E7004D291D292D0D02238
:101C9B00C0D075D008E5687003021D29E4F56475A2
:101CAB006701E56464086065E56425E0241BF58243
:101CBB00E4346FF583E0FEA3E08E65F566F4700304
:101CCB00E565F4603EE56955677015E5616566701D
:101CDB0004E56065657009E5674269AF6412270624
:101CEB00E5695567601DE5662401FFE43565FEEF88
:101CFB0065617003EE6560700AE567F45269AF6465
:101D0B001227960564E56725E0F5678095C3E52501
:101D1B0078D496E52418965005A62408A625E568E0
:101D2B0014601614601814601A24F96011146013EF
:101D3B00240B70121212E9800D121D54800812210F
:091D4B00188003122CD0D0D02224
:10291E00CBEFCBEBFD7C007E3A7F98120436CDEBED
:10292E00CD7C001204228E1A8F1B74002FF582EEBE
:10293E003434AF82F5188F197E347F008E1C8F1DB4
:09294E008E1E8F1FD213C2142249
:1029C900201933C213051FE51FAC1E7002051E1422
:1029D900F5828C83EFF0E51F65197004E51E651813
:1029E9007006751E34751F00E51F651D7004E51E10
:0729F900651C7002D21422DC
:102A6A00C214051DE51DAE1C7002051C14F5828EEC
:102A7A0083E0FFE51D65197004E51C65187006758D
:102A8A001C34751D00E51F651D7004E51E651C706C
:042A9A0002D213222F
:102ACE00C3E51F9FF51DE51E9EF51CC3E51D940075
:102ADE00E51C9434400BD3E51D9519E51C95184063
:0E2AEE000CE51B251DF51DE51A351CF51C22F7
:101A2C002573202562752025627520257520257566
:101A3C00202562752025627520256320256275207E
:101A4C0025632025632025630D0A00632069676EDA
:101A5C0020257520257520257520257520257520B8
:101A6C0025752025752025750D0A006320786D6974
:101A7C007420257520256275202562750D0A00637A
:101A8C0020677073202562750D0A00696E64657895
:101A9C00006572617365006F6666006F6E002A5692
:101AAC00455253494F4E3A20522D44415320563300
:101ABC002E320D0A0063210063207264617300638F
:101ACC002069676E006320786D697400632067700D
:101ADC007300633F00630063200067707320007223
:101AEC0065736574002A453A20756E6B6E6F776E60
:071AFC0020636D640D0A0078
:08000300E4F57DC216C21522CE
:1008F900906EDEEBF0A3EAF0A3E9F0300B13300CB5
:1009090008906EFB7401F0800D906EFB7402F0800C
:1009190005E4906EFBF0906EDEE0FBA3E0FAA3E045
:10092900F91203BA643F60030209D1906EE1E0F95C
:10093900A3E0FAA3E0906F30C9F0A3EAF0A3E9F0CD
:10094900906F09E0906F33F0906F08E0906F34F08A
:10095900906F04E0FFA3E0906F35CFF0A3EFF09024
:100969006F10E0FFA3E0906F37CFF0A3EFF0906F27
:1009790018E0906F39F0906F19E0906F3AF0300FEE
:10098900047F3180027F30906F3BEFF0906EFBE087
:10099900906F3CF03010047F3180027F30906F3DC2
:1009A900EFF0300E047F3180027F30906F3EEFF020
:1009B900300D047F3180027F30906F3FEFF07BFF75
:1009C9007A1A792C1200C922906EDEE0FBA3E0FAB4
:1009D900A3E0F91203BAFF122E12500C906EDFE455
:1009E90075F0011204C180E0E4906EFAF0906EDEB9
:1009F900E0FBA3E0FAA3E0F912142D906EFAE025CA
:100A0900E024E4F582E4346EF583EEF0A3EFF09090
:100A19006EDEE0FBA3E475F0011204D7A9F0FA1227
:100A290003BAFF122E1250E7906EFAE004F0E0B418
:100A39000BBB906EE5E0906F09F0906EE7E0906F68
:100A490008F0906EE8E0FFA3E0906F04CFF0A3EF09
:100A5900F0906EEAE0FFA3E0906F10CFF0A3EFF003
:100A6900906EEDE0906F18F0906EEFE0906F19F0D6
:100A7900906EF0E0FEA3E0FFEE4F24FF920FA3E09B
:100A8900FEA3E0FFEE4F24FF920BEF64014E7003CB
:100A9900D38001C3920C906EF4E0FEA3E0FFEE4F09
:100AA90024FF9210A3E0FEA3E0FFEE4F24FF920E75
:0D0AB900A3E0FEA3E0FFEE4F24FF920D220C
:10163E00906EDEEBF0A3EAF0A3E9F01203BA643F7A
:10164E0060030216D57BFF7A1A7957906F1BE0FF65
:10165E00A3E0906F30CFF0A3EFF0906F1DE0FFA3EB
:10166E00E0906F32CFF0A3EFF0906F1FE0FFA3E09A
:10167E00906F34CFF0A3EFF0906F21E0FFA3E090D6
:10168E006F36CFF0A3EFF0906F23E0FFA3E0906FE3
:10169E0038CFF0A3EFF0906F25E0FFA3E0906F3A04
:1016AE00CFF0A3EFF0906F27E0FFA3E0906F3CCF59
:1016BE00F0A3EFF0906F29E0FFA3E0906F3ECFF024
:1016CE00A3EFF01200C922906EDEE0FBA3E0FAA3B6
:1016DE00E0F91203BAFF122E12500C906EDFE47571
:1016EE00F0011204C180E0E4906EE1F0906EDEE055
:1016FE00FBA3E0FAA3E0F912142D906EE1E025E0D1
:10170E00241BF582E4346FF583EEF0A3EFF0906EB8
:10171E00DEE0FBA3E475F0011204D7A9F0FA120380
:10172E00BAFF122E1250E7906EE1E004F0E0B4081A
:02173E00BB22CC
:101BD700906EDEEBF0A3EAF0A3E9F01203BAB43F8C
:101BE700297BFF7A1A7977906F0BE0FFA3E0906F5C
:101BF70030CFF0A3EFF0906F15E0906F32F0906F59
:101C07002CE0906F33F01200C922906EDEE0FBA348
:101C1700E0FAA3E0F91203BAFF122E12500C906EED
:101C2700DFE475F0011204C180E0E4906EE7F09004
:101C37006EDEE0FBA3E0FAA3E0F912142D906EE745
:101C4700E025E024E1F582E4346EF583EEF0A3EFBE
:101C5700F0906EDEE0FBA3E475F0011204D7A9F063
:101C6700FA1203BAFF122E1250E7906EE7E004F063
:101C7700E0B403BB906EE1E0FFA3E0906F0BCFF001
:101C8700A3EFF0906EE4E0906F15F0906EE6E090B1
:041C97006F2CF0229C
:1024E400906EDEEBF0A3EAF0A3E9F0906EDEE0FB81
:1024F400A3E0FAA3E0F91203BAB43F127BFF7A1AFD
:10250400798B906F0AE0906F30F01200C922906EC0
:10251400DEE0FBA3E0FAA3E0F91203BAFF122E12E5
:10252400500C906EDFE475F0011204C180E0906EEF
:10253400DEE0FBA3E0FAA3E0F912142D906F0AEF9A
:02254400F02283
:1006F9007B017A6E799A7D20122CEC906EE1EBF0F9
:10070900A3EAF0A3E9F04A70047F0180027F009018
:100719006EEEEFF0605F7B017A6E799912142DC845
:10072900ECC8C9EDC9CAEECACBEFCB906F16E0FE93
:10073900A3E0FFE4FCFD1204EDC8ECC8C9EDC9CA89
:10074900EECACBEFCB906F06E0FEA3E0FFE4FCFD21
:10075900EB2FFFEA3EFEED39FDEC38FC906EE4121A
:100769000644906F16E0FEA3E0FFE4FCFD906EE8FE
:1007790012064480767B017A6E799912142DC8ECA1
:10078900C8C9EDC9CAEECACBEFCB906F12E0FFE43E
:10079900FCFDFE1204EDC8ECC8C9EDC9CAEECACB0E
:1007A900EFCB906F06E0FEA3E0FFE4FCFDEB2FFF2B
:1007B900EA3EFEED39FDEC38FC906EE412064490F9
:1007C9006EE1E0FBA3E0FAA3E0F912142DC8ECC82E
:1007D900C9EDC9CAEECACBEFCB906F12E0FFE4FCBA
:1007E900FDFE1204ED906EE8120644906EE4E0FC02
:1007F900A3E0FDA3E0FEA3E0FF780F1206318F7896
:10080900906EE4E0FCA3E0FDA3E0FEA3E0FFEE545C
:100819007FFEE48E768F77122E4F906EEEE06009A0
:10082900E4906EECF0A3F0800B120026906EECEED3
:10083900F0A3EFF0E4906EDEF0A3F0906EDEE0FE40
:10084900A3E0FFE4FCFD906EE8E0F8A3E0F9A3E083
:10085900FAA3E0FBC3120620606C122EC0906EE072
:10086900EFF0906EEEE06014906EE0E0FF906EEDB8
:10087900E02FF0906EECE03400F08018906EECE020
:10088900FEA3E0FF906EE0E0FD121FAD906EECEE6E
:10089900F0A3EFF0906EE0E0FF122F0C0577E577FB
:1008A900700205767004E57664807009F576F5774F
:1008B9000578122E4F906EDFE004F07006906EDE20
:1008C900E004F0020844906EEEE07013906EECE0E4
:1008D900FEA3E0FF122F32906EECEEF0A3EFF09042
:1008E9006EECE0FF122F0C906EEDE0FF122F0C2240
:102E2700D3EF648094B95007EF24D0FEFF8004EFFE
:042E370024A9FF22A9
:10183D00906EDEEBF0A3EAF0A3E9F0906EE574FF95
:10184D00F0A3741AF0A37497F0A3E4F0A37405F059
:10185D0012241AEF700312274E906EE574FFF0A359
:10186D00741AF0A3749DF0A3E4F0A37405F0906EC8
:10187D00DEE0FBA3E0FAA3E0F912241AEF700412E4
:10188D002D5722906EE574FFF0A3741AF0A374A384
:10189D00F0A3E4F0A37403F0906EDEE0FBA3E0FA96
:1018AD00A3E0F912241AEF7003C21522906EE574AD
:1018BD00FFF0A3741AF0A374A7F0A3E4F0A37402CD
:1018CD00F0906EDEE0FBA3E0FAA3E0F912241AEF2C
:1018DD007003D21522906EDEE0FBA3E0FAA3E0F9CF
:1018ED001203BAFF122B795043906EDEE0FBA3E09A
:1018FD00FAA3E0F99000011203D3FF122E27CDEFCA
:10190D00CD906EDEE0FBA3E0FAA3E0F91203BAFF7F
:10191D00122E27EFC454F02DFF906EE1F0122D889A
:0D192D00906EDFE475F0021204C180A92263
:042F6900122C1022F4
:0A2EE4007BFF7A1A79AA1200C922B6
:100AC600906EE574FFF0A3741AF0A374C1F0A3E46A
:100AD600F0A37402F07B017A6E799812241AEF70F3
:100AE60004120E4F22906EE574FFF0A3741AF0A361
:100AF60074C4F0A3E4F0A37406F07B017A6E7998CF
:100B060012241AEF7018906EE174FFF0A3741AF0B5
:100B1600A374C4F07B017A6E799E1208F922906E56
:100B2600E574FFF0A3741AF0A374CBF0A3E4F0A36A
:100B36007405F07B017A6E799812241AEF700A7B9D
:100B4600017A6E799D12163E22906EE574FFF0A32F
:100B5600741AF0A374D1F0A3E4F0A37406F07B0139
:100B66007A6E799812241AEF700A7B017A6E799E52
:100B7600121BD722906EE574FFF0A3741AF0A374CB
:100B8600D8F0A3E4F0A37405F07B017A6E7998128D
:100B9600241AEF700A7B017A6E799D1224E4229062
:100BA6006EE574FFF0A3741AF0A374DEF0A3E4F00C
:100BB600A37402F07B017A6E799812241AEF7018EA
:100BC600906EE174FFF0A3741AF0A374E1F07B0158
:100BD6007A6E79991208F922906EE574FFF0A37483
:100BE6001AF0A374E3F0A3E4F0A37402F07B017A95
:100BF6006E799812241AEF7018906EE174FFF0A3C4
:100C0600741AF0A374E1F07B017A6E79991208F9EF
:100C160022906E98E0B464041206F922906EE57490
:100C2600FFF0A3741AF0A374E6F0A3E4F0A374042F
:100C3600F07B017A6E799812241AEF700A7B017A9A
:100C46006E799C12183D22906EE574FFF0A3741A1B
:100C5600F0A374EBF0A3E4F0A37405F07B017A6EC5
:100C6600799812241AEF7004122F6922906E98E078
:100C7600B47604122EE422906E98E060097BFF7A27
:070C86001A79F11200C922E6
:102CB20010160280107568047F01122F147F1E12F5
:0E2CC2002E75120AC63015E81225A880E322EE
:102A0000C0D0EF20E72CEF640A6027EF640D60115F
:102A10007498257DF582E4346EF583EFF0057D80B2
:102A2000117498257DF582E4346EF583E4F0D216B6
:052A3000F57DD0D0226D
:102349002A4D4553534147453A2053746F72696E7C
:102359006720706172616D657465727320696E20A2
:10236900464C4153480D0A002A4D455353414745B0
:102379003A2046696E69736865642073746F72697F
:102389006E670D0A00000001C001C802000C001BA5
:102399000100193C03FFFFFFFFFFFFFFFFFFFFFFE6
:0A23A900FFFFFFFFFF00000A010024
:0A2EEE00757923757A8E12117B228C
:10117B0090238EE49324FF920BA3E49324FF920C11
:10118B00A3E49324FF9210A3E493906F08F09023B1
:10119B0092E49324FF920FE4906F12F07F80EF6044
:1011AB0014906F08E05F6007906F12E02402F0EF7D
:1011BB00C313FF80E9300F06906F12E004F0902309
:1011CB0093E493906F09F0902394E493906F0FF056
:1011DB00902395E493FF740193906F04CFF0A3EFEA
:1011EB00F0902397E493FF740193906F10CFF0A3CB
:1011FB00EFF0906F09E0FBFD7C007E037FE81204AB
:10120B0036906F13EEF0A3EFF0906F12E0FA8BF0C5
:10121B00A4FF906F16E5F0F0A3EFF0EB1313543F20
:10122B00906F1AF0FB906F2BF0902399E49324FFAF
:10123B00920EA3E49324FF920DA3E493906F18F006
:10124B0090239CE493906F19F090239DE493906FFF
:10125B0003F0906F0FE0FF7E00906F16E0FCA3E0B1
:10126B00FD120422906F06EEF0A3EFF0EBFF7E0071
:10127B00EAFD7C00120422E02F906F0EF0906F06B7
:10128B00E03E906F0DF0E4FFEF25E0249EF582E445
:10129B003423F583E493FC740193FDEF25E0241BC9
:1012AB00F582E4346FF583ECF0A3EDF00FEFB408A7
:1012BB00D79023AEE493FF740193906F0BCFF0A301
:1012CB00EFF09023B0E493906F15F09023B1E4937B
:0E12DB00906F2CF09023B2E493906F0AF022F3
:100E4F00A20BE433857A82857983F0A20CE433A375
:100E5F00F0A210E433857A82857983A3A3F0906F93
:100E6F0008E0857A82857983A3A3A3F0A20FE433E8
:100E7F00FFE57A2404F582E43579F583EFF0906F7E
:100E8F0009E0FFE57A2405F582E43579F583EFF083
:100E9F00906F0FE0FFE57A2406F582E43579F5834C
:100EAF00EFF0906F04E0FEA3E0FFE57A2407F582F0
:100EBF00E43579F583EEF0A3EFF0906F10E0FEA329
:100ECF00E0FFE57A2409F582E43579F583EEF0A3A6
:100EDF00EFF0A20EE433FFE57A240BF582E43579C7
:100EEF00F583EFF0A20DE433FFE57A240CF582E4ED
:100EFF003579F583EFF0906F18E0FFE57A240DF563
:100F0F0082E43579F583EFF0906F19E0FFE57A24ED
:100F1F000EF582E43579F583EFF0906F03E0FFE58E
:100F2F007A240FF582E43579F583EFF0E4906EDEE5
:100F3F00F0906EDEE0FF6408603BEF25E0241BF5C8
:100F4F0082E4346FF583E0FEA3E0FFE57A2410F529
:100F5F0082E43579F583C083C082906EDEE0D08263
:100F6F00D08375F002120681EEF0A3EFF0906EDEE3
:100F7F00E004F080BC906F0BE0FEA3E0FFE57A2465
:100F8F0020F582E43579F583EEF0A3EFF0906F153D
:100F9F00E0FFE57A2422F582E43579F583EFF090CE
:100FAF006F2CE0FFE57A2423F582E43579F583EFA2
:100FBF00F0906F0AE0FFE57A2424F582E43579F5A5
:100FCF0083EFF07BFF7A2379491200C9122A357B10
:090FDF00FF7A2379711200C92286
:101E9200E5C520E3FB75C50675C50EE5C530E4FB57
:101EA200AFC6EF75F004A4FFAEF0E5C5C41313543A
:101EB200037C002FF54DEC3EF54CE5C520E3FB75A8
:101EC200C50775C50FE5C530E4FBAFC6EF75F00475
:101ED200A4FFAEF0E5C5C4131354037C002FF54AEA
:101EE200EC3EF549F54E854A4FD21AE4F547F548DE
:101EF200FFEF25E02477F582E4346FF583E54CF0BB
:101F0200A3E54DF0E54D2548F548E54C3547F54745
:101F12000FEFB410DCE4F54BE5482401F54DE43550
:041F220047F54C2211
:10254600301A5EE5482401F54DE43547F54CE54B78
:1025560025E02477F582E4346FF583E0FEA3E0FFFF
:10256600C3E5489FF548E5479EF547E54B25E0243A
:1025760077F582E4346FF583E541F0A3E542F0E5B3
:10258600422548F548E5413547F547054BE54BB447
:102596001003E4F54B85494E854A4F852449852528
:0225A6004A22C7
:102D3D00C21B43878075985AE589540F4420F58945
:0A2D4D00758DFFD28ED2BCD2AC22ED
:03002300022B2786
:102B2700C0E0C0F0C083C082C0D075D01030980715
:102B3700AF99C298122A00309904C299D21BD0D0FB
:092B4700D082D083D0F0D0E0323E
:082F0C008F99301BFDC21B224E
:072F2400CEEFCE122F0C22AC
:102B5000E5C520E3FB8FC5EF4408F5C5E5C530E4C6
:102B6000FBAFC6EF75F004A4FFAEF0E5C5C41313C8
:092B70005403FDE5F0EF4DFF22D6
:102C1000E4F5A8F5E8F5B8F5F875780FE578A2E0E1
:102C200092B5A2E192B3A2E292B4A2E392B202FF01
:022C3000FE2282
:102E4F00E578A2E092B5A2E192B3A2E292B4A2E336
:032E5F0092B2220A
:0C2EC000E5764480857782F583E0FF22F0
:10002E0090D3557499F090ACAA7466F090D3557431
:10003E0090F0E575F5F0E576D2E7F583E577F58294
:0D004E00E5F0F0E0A2E730F701B340F72243
:10295700E578A2E092B5A2E192B3A2E292B4A2E333
:1029670092B290D3557499F090ACAA7466F090D354
:10297700557480F090D3557499F090ACAA7466F0B2
:092987009080007414F0D21C22AF
:102E6200301C0D908000E020E703D38001C3921C48
:032E7200A21C227D
:102A350075780C122957122E6240FB75780D122EEF
:102A45004FE4F576F577857782857683E0F575121F
:102A5500002E0577E57770020576E5777004E57653
:052A6500648070E22214
:032F7900C21C2255
:03005B000222DDA1
:1022DD00C0E0C0D0C2CC742D25C9F5C93017581532
:1022ED0050E5507052E55670128552FCC2C0F55142
:1022FD00755601E55425E0F550803CE556640170B6
:10230D002375FCFFD2C00551E5516553700E301891
:10231D0007F556855550801FC217801B75560275DF
:10232D0050028013E556B4020E8552FCC2C075569C
:0C233D0001E55425E0F550D0D0D0E0328E
:102D700075FCFFD2C075FE0B75528075EA0DC2FC62
:082D8000D2EC75550AC21722BE
:102BCA00C217A202921875FCFFD2C08F53E4F556C1
:102BDA00CEEDCE8EFECEEBCE8E54855550EF6002F2
:032BEA00D21722DD
:062F3900D202122BCA2295
:062F3F00C202122BCA229F
:082F14007D0B7B01122F392215
:082F1C007D327B04122F3922E3
:102E7500C21775FCFFD2C08F55E4F556855550D263
:022E8500172212
:101B03002A4D3A20615F7374203D2025750D0A002C
:101B13002A4D3A2061283029203D2025750D0A00E1
:101B23002A573A20615F73743D25752C2061303D3F
:101B330025752028672D73772064697361626C654E
:101B430064290D0A002A4D3A2070283029203D20AF
:101B530025750D0A002A573A20502072616E676579
:101B6300205B25752C25755D0D0A002A573A204206
:101B730057206572726F722028425720646973611F
:101B8300626C6564290D0A002A573A206E6F20693A
:101B9300676E202562640D0A002A573A206E6F2073
:101BA300786D69740D0A002A573A206E6F206770AA
:101BB300730D0A002A573A2064726F6775652065B2
:101BC30072720D0A002A573A206D61696E206572A0
:041BD300720D0A0085
:072F2B00EF60031F80FA2292
:102C9300A2029293E4F57BF57C7F78122F2B057CBF
:0F2CA300E57C7002057BE57C640A457B70EB22C3
:100FE800E4906EE3F0906EDEF0A3F0906EE2F0D243
:100FF80002122C937F06122B50906EDFE02FF09098
:101008006EDEE03EF0C202122C93906EE2E004F035
:10101800E0B420DB906EDEE0FEA3E0FF7C007D20E4
:1010280012048B906EDEEEF0A3EFF07BFF7A1B7953
:1010380003906F30EEF0A3EFF01200C9E4906EE079
:10104800F0A3F0A3F07F06122B50906EE1E02FF092
:10105800906EE0E03EF0906EE2E004F0E0B420E54F
:10106800906EE0E0FEA3E0FF7C007D2012048B90F0
:101078006EE0EEF0A3EFF07BFF7A1B7913906F30F0
:10108800EEF0A3EFF01200C9906EE0E0FEA3E0FFDF
:10109800906EDEE0FCA3E0FDC39FFFEC9EFEC3EF75
:1010A800942DEE64809480502D7BFF7A1B792390D9
:1010B8006F30ECF0A3EDF0906EE0E0FFA3E0906FEE
:1010C80032CFF0A3EFF01200C97F06122F1CC21016
:1010D800906EE37406F0E4906EDEF0A3F0906EE29A
:1010E800F07F07122B50906EDFE02FF0906EDEE05D
:1010F8003EF0906EE2E004F0E0B420E5906EDEE0B1
:10110800FEA3E0FF7C007D2012048B906EDEEEF0E3
:10111800A3EFF07BFF7A1B7948906F30EEF0A3EFD6
:10112800F01200C9906EDEE0FEA3E0FFC3947DEEEE
:1011380064809482400BD3EF94DBEE648094834008
:101148002C7BFF7A1B7958906F30EEF0A3EFF0A359
:101158007402F0A3747DF0A37403F0A374DBF0129F
:1011680000C97F05122F1C906EE37405F0906EE3A2
:03117800E0FF2273
:10193A00E4906EDEF0300B1EA294300C01B3401618
:10194A007BFF7A1B796E1200C97F03122F1CC20B10
:10195A00906EDE7403F0E4906EDFF0906EDFE0FFCD
:10196A006408606AEF25E0241BF582E4346FF5838E
:10197A00E0FCA3E0F47002ECF4604B122ECC401FA2
:10198A007F04122F1C7BFF7A1B798B906EDFE00499
:10199A00906F30F01200C9906EDE7404F0802790C8
:1019AA006EDFE0FF1226BA401D7F04122F1C7BFF58
:1019BA007A1B798B906EDFE004906F30F01200C9C9
:1019CA00906EDE7404F0906EDFE004F0808D906F0C
:1019DA000BE07002A3E06020122F4B401B7F041221
:1019EA002F1C7BFF7A1B799C1200C9E4906F0BF0C5
:1019FA00A3F0906EDE7404F0906F0AE0601E122F5E
:101A0A004540197F04122F1C7BFF7A1B79AA12000A
:101A1A00C9E4906F0AF0906EDE7404F0906EDEE016
:021A2A00FF2299
:10299000D20112193A906FB5EFF06002C201120F26
:1029A000E8906FB6EFF06002C20120C60B7BFF7AA1
:1029B0001B79B71200C9C20120C70B7BFF7A1B79B4
:0929C000C81200C9C201A20122E3
:10000E00E4FF74B12FF582E4346FF58374FFF00FC3
:05001E00EFB404EE2226
:0C2ECC00EFC31325E02441FF122D082263
:1026BA00906EE0EFF0E0FFC31325E02441FF7B01B9
:1026CA007A6E79E2906EE87401F0122864906EE1F5
:1026DA00EFF0906EE0E054012402FF74017E00C81E
:1026EA00EFC8088005C333CE33CED8F9FF906EE227
:0C26FA00E0FDE4EF5D6003D38001C3222B
:10270600CEEFCEEEC313FF24B1F582E4346FF5832A
:10271600C083C082E0FDEE5401FC7401C8ECC80819
:102726008002C333D8FCF45DD082D083F0EF25E07D
:102736002440FFEEC31324B1F582E4346FAD82FC6E
:082746007B01D2011228E322FD
:10279600CEEFCEEEC313FF24B1F582E4346FF5839A
:1027A600C083C082E0FDEE5401FC7401C8ECC80889
:1027B6008002C333D8FC4DD082D083F0EF25E024CD
:1027C60040FFEEC31324B1F582E4346FAD82FC7B87
:0727D60001D2011228E322E9
:102DFC00E4F57EFF746A2FF582E4346FF583E4F01A
:062E0C000FEFB40DEF22F0
:062F45007F50122D08224E
:102D8800906EE2EFF07F507C6E7DE27B01D2011203
:082D980028E3906EE3EFF02246
:1025A8007F537B017A6E79DF906EE87401F0122810
:1025B80064906EDEEFF0A3E0D3941040037410F043
:1025C800906EDFE0FE603A7F517B017A6F799790D9
:1025D8006EE8F0122864906EDEEFF0E4F0906EDFA3
:1025E800E0FF906EDEE0FE6F601774972EF582E4D0
:1025F800346FF583E0FF122F0C906EDEE004F0805C
:02260800DC22D2
:10274E00E4906EE2F07F577B017A6F7997906EE896
:10275E007410F0122864906EE3EFF0E4F0906EE3E4
:10276E00E0FF6410601774972FF582E4346FF583E1
:10277E00E0FF122F24906EE3E004F080E0906EE212
:08278E00E004F0E0B408BE22F3
:102D5700906EE27442F07F567C6E7DE27B01D20179
:092D67001228E3906EE3EFF02264
:102DA000906ED9EFF07F547C6E7DD97B01C2011209
:082DB00028E3906EDAEFF02237
:102A9E00C0D075D008906F0AE06022057E906F0955
:102AAE00E0657E7018F57E7F557B017A6F796490B4
:102ABE006EE8740DF0122864906ED8EFF0D0D0222C
:1020A200D21DE4F557F558F559906F09E0FF75F028
:1020B2000A84755C00F55DEFC313755A00F55B90F9
:1020C2006F0BE0FEA3E0FF4E604B906F557404F07F
:1020D200E4A3F0FCFDF8F9CAEECACBEFCBFF7EC059
:1020E2007DA81227DD7B107A00790078001227DDA7
:1020F200EF14906F57F0906F2CE075F080A4FF9072
:102102006F15E02F906F58F07F607C6F7D557B04D8
:06211200D2011228E322B5
:062F4B007F60122D082238
:1023B300C0E0A3E558F0A3E559F0A3E52AF0A3E5AF
:1023C3002CF0A3E52EF0A3E530F0A3E532F0A3E56E
:1023D30034F0A3E536F0A3E538F0A375F000E52962
:1023E30042F0E52B232342F0E52DC442F0E52FC450
:1023F300232345F0F0A375F000E53142F0E53323E4
:102403002342F0E535C442F0E537C4232345F0F019
:07241300A3E540F0D0E02238
:101DF500C0D075D008906F0BE07002A3E0700302AD
:101E05001E8F301D09E5686005E4F557C21DE557CD
:101E1500FB7A00AC5CAD5DFFCEEACE120436ED4C2C
:101E2500705C906F0AE0601DAC5AAD5BCFEBCFCE16
:101E3500EACE120436ED4C700C906ED8741CF0A3EB
:101E45007402F0800A906ED8740FF0A37401F090BC
:101E55006ED8E0906F55F0906ED9E0906F56F01205
:101E650023B37F607C6F7D55906ED8E0FBC2011275
:101E750028E3E56860080559E559700205580557D6
:0D1E8500906F09E065577002F557D0D0222C
:102C53000000CC01D8011400F0013C002800E4017D
:102C6300A0016C007800B40150009C01880144006D
:050026007EFF7FFF22B8
:101FAD00CBEFCBCAEECAC9EDC9E9540FFFEAEB6F0F
:101FBD00540F25E0FFE433FE74532FF582EE342CDD
:101FCD00F583EAC4F854F0C868FEEBC4540F48FF1B
:101FDD00EE540FFEE4936EFA7401936FFBCFE9CFCD
:101FED00EFC4540F540FFFEAEF6B540F25E0FFE4DD
:101FFD0033FE74532FF582EE342CF583EAC4F85476
:10200D00F0C868FEEBC4540F48FFEE540FFEE49386
:0C201D006EFA7401936FFBCEEACEFF2236
:072F3200EEF4FEEFF4FF22B4
:10260A00FF2F6DFF2EF8FF2F02FF2C32FF2F51FFF5
:10261A002BEDFF2F57FF2F71FF2DB8FF2F5DFF2CDA
:10262A0073FF2E3BFF2F75FF2F7CFF2F7DFF2F7E21
:10263A00FF2F7FFF2F80FF2F81FF2F82FF2F83FF26
:10264A002F84FF2F85FF2F86FF2F87FF2F88FF2FCD
:10265A0063FF2F63FF2F63FF2F63FF2F63FF2F6338
:0F2E9800D296D29775D8C575DBECD2BDD2AD22DC
:102D0800E4F56F8F6DD21ED2DDFF122AFCEF641836
:0B2D18006004EFB44003D38001C3222D
:1028E300906EE4ECF0A3EDF08C838D82787FEBFEA9
:1028F3006006E0F6A308DEFA8B6F8F6DD21ED2DD81
:1029030030010DCFEBCF122AFC906EE6EFF080057D
:0B291300E4906EE6F0906EE6E0FF221C
:10286400906EE5EBF0A3EAF0A3E9F0CEEFCEA3E09F
:10287400FFF56F8E6DD21ED2DD122AFCE4FE906E3F
:10288400E8E06E601D747F2EF8E6FD906EE5E0FBD7
:10289400A3E0FAA3E0F98E82758300ED1204000E22
:0328A40080DC22B3
:102AFC00CEEFCEE4F56AEE2402FDE433FCE56A6D1C
:102B0C007001EC6010756BDDD56BFD201E03AF6E94
:0B2B1C0022056A80E175D8D57F0022F9
:042F6D0075D8D5221C
:0A2EF800856DDA75D8C5E4F56C228B
:0A2F0200856DDA75D8C5E4F56C2280
:102C3200C0D075D010E56F700775D8D5C21E800E52
:102C4200AF6C056C747F2FF8E6F5DA75D8C5D0D075
:012C5200225F
:062F510075D8D5C21E2256
:102BED00C0D075D010E56C656F700775D8D5C21E55
:102BFD00800EAF6C056C747F2FF8E6F5DA75D8C5CD
:032C0D00D0D02202
:062F570075D8D5C21E2250
:042F710075D8E52208
:102DB800E56F14600A04700C75D8D5C21E800875BA
:082DC800D8C1800375D8C522B3
:062F5D0075D8D5C21E224A
:102C7300C0D075D010747F256CF8A6DAE56F140503
:102C83006C656C700575D8C1800375D8C5D0D0222A
:102E3B00C0D075D010747F256CF8A6DA75D8D5C2C2
:042E4B001ED0D022A3
:042F750075D8D52214
:012F7C002232
:012F7D002231
:012F7E002230
:012F7F00222F
:012F8000222E
:012F8100222D
:012F8200222C
:012F8300222B
:012F8400222A
:012F85002229
:012F86002228
:012F87002227
:012F88002226
:062F630075D8D5C21E2244
:03002B000228A701
:1028A700C0E0C0F0C083C082C0D075D01085D96E9B
:1028B700E5D9131313541F75F003A4240AF582E412
:1028C7003426F583E493740193FA740293F912069C
:0C28D7008DD0D0D082D083D0F0D0E03281
:03000000022ED8F5
:0C2ED800787FE4F6D8FD7581D6021F2635
:1003BA00BB010689828A83E0225002E722BBFE0241
:0903CA00E32289828A83E4932274
:1003D300BB010CE58229F582E5833AF583E02250DF
:1003E30006E92582F8E622BBFE06E92582F8E22229
:0D03F300E58229F582E5833AF583E4932243
:10040000F8BB010DE58229F582E5833AF583E8F032
:10041000225006E92582C8F622BBFE05E92582C8DE
:02042000F222C6
:10042200EFF88DF0A4FFEDC5F0CEA42EFEEC88F01F
:04043200A42EFE22D4
:10043600BC000BBE0029EF8DF084FFADF022E4CCAA
:10044600F875F008EF2FFFEE33FEEC33FCEE9DEC73
:10045600984005FCEE9DFE0FD5F0E9E4CEFD22EDB9
:10046600F8F5F0EE8420D21CFEADF075F008EF2F03
:10047600FFED33FD4007985006D5F0F222C398FDF4
:050486000FD5F0EA2291
:10048B00C2D5EC30E709B2D5E4C39DFDE49CFCEE8C
:10049B0030E715B2D5E4C39FFFE49EFE120436C3CA
:1004AB00E49DFDE49CFC800312043630D507C3E4C5
:0604BB009FFFE49EFE22FB
:1004C100C5F0F8A3E028F0C5F0F8E58215827002C6
:0604D1001583E038F02263
:1004D700A3F8E0C5F025F0F0E582158270021583D8
:0604E700E0C838F0E82235
:1004ED00E88FF0A4CC8BF0A42CFCE98EF0A42CFCAE
:1004FD008AF0EDA42CFCEA8EF0A4CDA8F08BF0A42C
:10050D002DCC3825F0FDE98FF0A42CCD35F0FCEB8A
:10051D008EF0A4FEA9F0EB8FF0A4CFC5F02ECD394F
:0F052D00FEE43CFCEAA42DCE35F0FDE43CFC22BC
:10053C0075F008758200EF2FFFEE33FECD33CDCC76
:10054C0033CCC58233C5829BED9AEC99E5829840F9
:10055C000CF582EE9BFEED9AFDEC99FC0FD5F0D6D6
:10056C00E4CEFBE4CDFAE4CCF9A88222B800C1B900
:10057C000059BA002DEC8BF084CFCECDFCE5F0CB3E
:10058C00F97818EF2FFFEE33FEED33FDEC33FCEB77
:10059C0033FB10D703994004EB99FB0FD8E5E4F932
:1005AC00FA227818EF2FFFEE33FEED33FDEC33FC1F
:1005BC00C933C910D7059BE99A4007EC9BFCE99A13
:1005CC00F90FD8E0E4C9FAE4CCFB2275F010EF2F58
:1005DC00FFEE33FEED33FDCC33CCC833C810D70758
:1005EC009BEC9AE899400AED9BFDEC9AFCE899F893
:0E05FC000FD5F0DAE4CDFBE4CCFAE4C8F92226
:1027DD00C2D5E830E70FB2D5E4C39BFBE49AFAE427
:1027ED0099F9E498F8EC30E717B2D51228131205D1
:1027FD0078E4C39BFBE49AFAE499F9E498F8800332
:10280D0012057830D50DE4C39FFFE49EFEE49DFDD7
:04281D00E49CFC2219
:10060A00EB9FF5F0EA9E42F0E99D42F0EC6480C867
:06061A0064809845F02207
:10062000EB9FF5F0EA9E42F0E99D42F0E89C45F030
:0106300022A7
:10063100E8600FECC313FCED13FDEE13FEEF13FFA7
:03064100D8F122CB
:0C064400ECF0A3EDF0A3EEF0A3EFF02229
:10065000A8828583F0D083D08212066712066712C3
:100660000667120667E473E493A3C583C5F0C583E8
:10067000C8C582C8F0A3C583C5F0C583C8C582C8F4
:010680002257
:0C068100A42582F582E5F03583F5832284
:06068D008A838982E473F8
:10005E00E5702430F582E4346FF583E0057022906C
:10006E006F2D300903906F30E475F0011206B30264
:10007E0003BA2002E97F2ED2028018EF540F24908B
:10008E00D43440D4FF30060BEF24BFB41A00500313
:10009E002461FFE571600215710574E57470020547
:1000AE007330090E906F2DE475F0011206B3EF0256
:1000BE000693022F247403D2098003E4C209F5705B
:1000CE00906F2D1206CAE4F571F573F574E5716043
:1000DE00077F201200A180F5F572C203C202C2048E
:1000EE00C205C207C208C20A12006DFF700D3009A8
:1000FE00057F001200B2AF74AE7322B42561C2D573
:10010E00C20612006DFF24D0B40A00501C75F00A0E
:10011E0020D50DC571A42571F5717002D20580E050
:10012E00C572A42572F57280D724CFB41A00EF5091
:10013E0004C2E5D2060202ACD20380C4D20280BE53
:10014E00D20480BAD2D580B8D20780B27F201200F6
:10015E00A12004077401B5710040F112005EFF1278
:10016E0000A10200DBD20AD208809312005EFB12BD
:10017E00005EFA12005EF94A4B700679787A037BBC
:10018E00FF200433E571602FAF72BF00011F7E00A8
:10019E008E827583001203D360050EEE6F70F1C26E
:1001AE00D5EBC0E0EAC0E0E9C0E0EE1202F0D0E02C
:1001BE00F9D0E0FAD0E0FB1203BAFF60A5EBC0E085
:1001CE00EAC0E0E9C0E01200A1D0E02401F9D0E0DD
:1001DE003400FAD0E0FBE57260DDD572DA80837B05
:1001EE00FF7A0279ECD2048098791080027908C2E5
:1001FE0008C20A8008D2D5790A8004790AC2D5E4E9
:10020E00FAFDFEFF12005EFC7B0820031312005E57
:10021E00FD7B1030020A12005EFE12005EFF7B2094
:10022E00EC3382D592D55013C3E43002069FFFE41F
:10023E009EFEE42003039DFDE49CFCE4CBF8C20388
:10024E00EC700CCFCECDCCE824F8F870F38017C349
:10025E00EF33FFEE33FEED33FDEC33FCEB33FB9966
:10026E004002FB0FD8E9EB300305F8D0E0C448B2EA
:10027E0003C0E00AEC4D4E4F78207B0070C2EAC0FE
:10028E00E01202F2D0F0D0E0200304C4C0E0C4B209
:10029E0003C0F012008AD0F0D5F0EB0200DB12069C
:1002AE00D301795301F758014A4C01464201FB4FE5
:1002BE00020344020349015F4302095501ED460161
:1002CE00ED4501ED47039B50014E2D01522E017558
:1002DE002B01562301732003862A0000016D3F3F38
:1002EE003F00790AA2D5200514300709B91002047F
:1002FE0004B9080104A2D5200802500104200466A6
:02030E00920457
:10031000B571005032C0E07F203005177F30A20455
:1003200072087207500D120347C204C208C2077F49
:1003300030800F300703E9C0E01200A1300703D07E
:10034000E0F9D0E0B571CE3007177F30B9100C124C
:1003500000A17F583006077F788003B90803120098
:10036000A13004057F2D0200A17F20200AF87F2BF9
:100370002008F322920480CF286E756C6C29002D22
:1003800050434958D20312005E3003F8C20378711B
:1003900030D504D2027872F602010C12005E2403FA
:1003A000B405004001E490037F93120092743A1266
:0A03B0000092D2057571040201F7F6
:102E1200EFC394094006EFC3940E4004EFB42003BD
:052E2200D38001C32272
:102B7900EFC394414006EFC394474018EFC39461F3
:102B89004006EFC39467400CEFC394304009EFC38C
:092B9900943A5003D38001C322D9
:10241A00906EE2EBF0A3EAF0A3E9F0906EE5E0FB40
:10242A00A3E0FAA3E0F91203BAFE906EE2E0FBA37E
:10243A00E0FAA3E0F91203BAFD6E702AED600E907D
:10244A006EE874FFF5F01204C145F070037F0022B4
:10245A00906EE3E475F0011204C1906EE6E475F043
:10246A00011204C180B5D3EE6480F8ED648098400F
:07247A00037F01227FFF2216
:102CEC00E94A4B7001221203BAFF6D700122EF709A
:0C2CFC0004FBFAF92209E970ED0A80EAF5
:10142D00906EFCEBF0A3EAF0A3E9F0906EFCE0FB0C
:10143D00A3E0FAA3E0F91203BAFF122E12500C909A
:10144D006EFDE475F0011204C180E0D201906EFCD6
:10145D00E0FBA3E0FAA3E0F91203BAFF642B6004EA
:10146D00EFB42D1D906EFCE0FBA3E475F0011204AA
:10147D00D7A9F0FA1203BA642D6003D38001C39289
:10148D0001906EFF12065000000000906EFCE0FB14
:10149D00A3E0FAA3E0F91203BAFF122E87506A7F78
:1014AD000A7E007D007C00906EFFE0F8A3E0F9A3BA
:1014BD00E0FAA3E0FB1204EDC8ECC8EDC0E0EEC00D
:1014CD00E0EFC0E0906EFCE0FBA3E0FAA3E0F912C0
:1014DD0003BAFF3395E0FEEF24D0FFEE34FFFEE4B8
:1014ED00FCFDD0E0FBD0E0FAD0E0F9EB2FFFEA3EB7
:1014FD00FEED39FDEC38FC906EFF120644906EFD4A
:10150D00E475F0011204C18082300110906EFFE08D
:10151D00FCA3E0FDA3E0FEA3E0FF8011906EFFE0D1
:0E152D00FCA3E0FDA3E0FEA3E0FF1206A52252
:10069300BB010689828A83F0225002F722BBFE0146
:0206A300F32240
:0E06A500C3E49FFFE49EFEE49DFDE49CFC2266
:1006B300F8E0FBA3A3E0F925F0F0E58215827002D0
:0706C3001583E0FA38F02274
:0906CA00EBF0A3EAF0A3E9F02231
:1006D300D083D082F8E4937012740193700DA3A3B6
:1006E30093F8740193F5828883E4737402936860CA
:0606F300EFA3A3A380DFCA
:102E8700EFC394304009EFC3943A5003D38001C392
:012E97002218
:00000001FF
